:020000020000FC
:0200000055C0E9
:0200240020C1F9
:02002800C5C24F
:02002C00E8C228
:1000AC00FF240AE00EBF0FEF0DBF00E800936100C4
:1000BC00002700936100569A579A869A859A849ADB
:1000CC005E9A4CD580E875D5FCE0E2EDA0D580ECCD
:1000DC0070D5FCE0E4EE9BD5BB27A3E055D25E982F
:1000EC000091C90008610093C90006E00093CA00A2
:1000FC0000270093CD0007E60093CC000027009367
:10010C00000100EC00937C0007E800937A0026982D
:10011C002E9A00E400936B000027009324013327F0
:10012C0000E300930D0500E300930E0500E300933C
:10013C000F0500E30093100500E70093110500E79D
:10014C00009312050DE60093130500E200931405CD
:10015C0000270093150500E30093220500E30093AC
:10016C0023050FED0093240503E40093250500E21D
:10017C000093260500270093270500E30093320522
:10018C0000E30093330505E2009334050027009348
:10019C00350552D27894B6D50E94EC0B0E94650AB4
:1001AC000E94A40A009136058BD161D10E94650A88
:1001BC000E94A40A10913605011711F40E94250B18
:1001CC000E94410B0E94650A0E94A40AC2E1D1E080
:1001DC00E4E3FCE1059109930D30E1F7009168052A
:1001EC0000931201009169050093130100916A05B7
:1001FC000093150100916B050093160100916C059D
:10020C000093180100916D05009319010EE4009301
:10021C00010100EC009302010027009303010E94EE
:10022C00390C00270093CD0009E10093CC0001E0CC
:10023C00009368008C9AABD5CAD72AD63F3FD1F72A
:10024C00332709B110E401270BB90E94650A0E94FB
:10025C00A40A8C980ED02AD0EDCF0F930FB70F9322
:10026C008D9A1E9B02C03FEF8D980F910FBF0F917F
:10027C0018958F93EF93FF9380E89BD4F5E0E1E51D
:10028C00CED48E9A80EC95D4F5E0EDE0C8D488EC11
:10029C0090D4F5E0E2E2C3D48DEC8BD4F5E0E2E34C
:1002AC00BED48E98FF91EF918F9108950F932F9359
:1002BC008F939F93AF93BF93CF93DF93EF93FF9362
:1002CC000E94630C803021F40027009324018DC020
:1002DC0000916705003311F00533C9F70091240133
:1002EC000130B9F0A0E0B3E0EAEFFBE12227059181
:1002FC000D93003019F02395FACF8E9A0E943F0D82
:10030C00209310010E945C0D0E94840D01E000936B
:10031C002401009168050093000300916905009386
:10032C0001030EE20093020300916A05009303039C
:10033C0000916B05009304030EE2009305030091FA
:10034C006C050093060300916D050093070309E00B
:10035C000093080300916205009309030091630563
:10036C0000930A030AE300930B03009164050093C6
:10037C000C030091650500930D030AE300930E0333
:10038C000091660500930F0300916705009310031D
:10039C0009E000931103A2E1B3E0C8E1D5E00991B3
:1003AC000D930F3DE1F709E000931803A9E1B3E0C9
:1003BC00CBE2D5E009910D930532E1F709E000930A
:1003CC001E03AFE1B3E0CDE0D5E009910D9300370A
:1003DC00E1F70DE0009323030E943F0D04E200932C
:1003EC0010010E945C0D0E94840DFF91EF91DF9132
:1003FC00CF91BF91AF919F918F912F910F910895B4
:10040C0000000000000000000000000000000000E0
:10041C00000008958F939F9380E190E00197F1F78E
:10042C009F918F9108958F939F9384E290E0019711
:10043C00F1F79F918F9108958F939F9384EC90E0A7
:10044C00019739F49F918F9108958F939F938CE826
:10045C0091E00197F1F79F918F9108958F939F935E
:10046C008CEC97E00197F1F79F918F9108958F9302
:10047C009F938CE99FE00197F1F79F918F910895DD
:10048C008F939F938CE19EE40197F1F79F918F914D
:10049C0008958F939F938CE39CE90197F1F79F91BB
:1004AC008F910895AF93AAE0F4DFAA95E9F7AF9185
:1004BC000895AF93A2E3EDDFAA95E9F7AF91089504
:1004CC00AF93A4E6E6DFAA95E9F7AF910895AF9351
:1004DC00BF93A4EFB1E0DDDF1197E9F7BF91AF91C6
:1004EC000895AF93BF93A8EEB3E0D3DF1197E9F76C
:1004FC00BF91AF910895AF93BF93A0E7B7E1C9DF68
:10050C001197E9F7BF91AF910895AF93BF93A0E610
:10051C00BAEEBFDF1197E9F7BF91AF910895AF9392
:10052C00BF936EDF1197E9F7BF91AF910895AF9329
:10053C00BF9379DF1197E9F7BF91AF910895AF930E
:10054C00BF9383DF1197E9F7BF91AF910895AA2369
:10055C0019F4BB2309F40895AF93BF9388DF119767
:10056C00E9F7BF91AF910895AF93BF9392DF1197C5
:10057C00E9F7BF91AF910895AF93BF9393DF1197B4
:10058C00E9F7BF91AF910895AF93BF9399DF11979E
:10059C00E9F7BF91AF910895AF93BF93ACDF11977B
:1005AC00E9F7BF91AF9108950F930FB70F93009197
:1005BC00E10003FF1AC00091E100077F0093E10006
:1005CC0000E00093000500E00093010500E00093BB
:1005DC00020500E00093030500E0009304054CD0F5
:1005EC000091F00008600093F0000F910FBF0F9185
:1005FC0018950F930FB70F930091F400013029F069
:10060C00023061F0043079F013C000E00093E9008F
:10061C000091E80003FF0CC059D00AC001E0009320
:10062C00E9007BD105C002E00093E9000AD200C0CA
:10063C000F910FBF0F9118950F9301E00093D70006
:10064C0000EB0093D80000E90093D80000EB009376
:10065C00D80000E109BD02E109BD09B500FFFDCFDD
:10066C0000E90093D80000270093E00008E0009315
:10067C00E20078940F9108950F931F930091000559
:10068C000093E9000091EB0001600093EB000091F6
:10069C00010507950795079510910205012B00930D
:1006AC00EC0000910305000F000F000F000F1091DC
:1006BC000405110F110F012B0093ED000091ED00BB
:1006CC0002600093ED001F910F9108950F931F93FB
:1006DC00EF93FF930091F100009305050091F10059
:1006EC00009306050091F100009307050091F100BD
:1006FC00009308050091F100009309050091F100A9
:10070C0000930A050091F10000930B050091F10094
:10071C0000930C050091E800077F0093E80000911E
:10072C000505007619F0003261F4A7C000910605AA
:10073C00003041F00530A9F0063039F1093009F4E8
:10074C0056C0A0C000270093F1000093F100009167
:10075C00E8000E7F0093E8000091E8000470E1F3DC
:10076C0096C0009107050F770093E3000091E80015
:10077C000E7F0093E8000091E8000170E1F3009116
:10078C00E30000680093E30082C00091080501308B
:10079C0039F0023041F0033059F0023201F177C0E8
:1007AC00EEEBFAE021C020910B05E0EDFAE01DC064
:1007BC0000910705003039F0013041F0023049F06A
:1007CC00033051F012C0EAEFFAE00EC0EEEFFAE09F
:1007DC000BC0E0E1FBE008C0ECE3FBE005C02091BE
:1007EC000B05E8E4FBE001C0249156D050C012E0A8
:1007FC001093E9000091EB000E7F0093EB00009149
:10080C00ED000D7F0093ED001A9591F701E0009338
:10081C00000503E00093010501E00093020503E0ED
:10082C000093030501E00093040526DF0091F0001E
:10083C0000640093F00002E00093000503E00093D5
:10084C00010500E00093020503E00093030501E0BD
:10085C000093040511DF0091F00004600093F00098
:10086C0000270093E9000091E8000E7F0093E80058
:10087C000091E8000170E1F30AC000910605013017
:10088C0009F405C00091EB0000620093EB00FF91AE
:10089C00EF911F910F9108950F931F9311270091C2
:1008AC00E800047031F505910093F1002A95139539
:1008BC0007E0012349F40091E8000E7F0093E80063
:1008CC000091E8000570E1F3203049F70091E80051
:1008DC00047009F009C00091E8000E7F0093E80055
:1008EC000091E8000470E1F30091E8000B7F0093A5
:1008FC00E8001F910F9108950F9300270093F100CA
:10090C000093F1000091E8000E7F0093E800009145
:10091C00E8000470E1F30F9108950F930091E80043
:10092C00007409F48CC00091E8000F7B0093E80080
:10093C000091E800017009F482C00091E8000E7F7C
:10094C000093E800009162050093F10000916305AB
:10095C000093F1000AE30093F10000916405009309
:10096C00F100009165050093F1000AE30093F1009A
:10097C00009166050093F100009167050093F1006A
:10098C00009168050093F100009169050093F10056
:10099C000FE20093F10000916A050093F1000091C1
:1009AC006B050093F1000FE20093F10000916C05D0
:1009BC000093F10000916D050093F10000910D057D
:1009CC000093F10000910E050093F10000910F05CA
:1009DC000093F100009110050093F10000911805AF
:1009EC000093F100009119050093F10000911A0594
:1009FC000093F10000911B050093F10000911C0580
:100A0C000093F10000911D050093F10000912B055E
:100A1C000093F10000912C050093F10000912D053D
:100A2C000093F10000912E050093F10000912F0529
:100A3C000093F1000091E8000F770093E8000F910C
:100A4C0008950F931F930091E800047079F10091C1
:100A5C00E8000B7F0093E8000091E800007231F190
:100A6C000091F100009336050091F10000933705D9
:100A7C000091F100009338050091F10000933905C5
:100A8C000091F10000933A050091F10000933B05B1
:100A9C000091F10000933C050091F10000933D059D
:100AAC00D8D40091E8000F770093E8001F910F91C4
:100ABC0008951201100100000008EB03050001006D
:100ACC00010203010902290001010080FA09040056
:100ADC000002030000000921100100012220000780
:100AEC0005810340000107050203400001000403D7
:100AFC0009041203570045004900470055002E0019
:100B0C004C0055002C035400450045004E0053008A
:100B1C005900200032002E0030002000480049000F
:100B2C0044002D00440065007600690063006500F8
:100B3C000C035700540048003100430006A0FF0985
:100B4C0001A101090315002540951F7508810209B3
:100B5C000415002540950875089102C00F938F93DA
:100B6C0004B10F6304B99EDC05B10360037C05B9C5
:100B7C001BD086DC05B10360037C05B915D005B12B
:100B8C000360037C05B910D005B10260027C05B985
:100B9C000BD088E20ED08FE00CD086E00AD08CE02F
:100BAC0008D08F910F9108952D9A4FDC2D9856DC1B
:100BBC0008950F931F93082F02950F7015B1102BEA
:100BCC00006F10231F7E15B9EFDF8F7015B1182B36
:100BDC00806F18231F7E15B9E7DF1F910F910895C1
:100BEC000F931F93082F02950F7015B1102B006FE8
:100BFC001023106115B9D8DF8F7015B1182B806FC9
:100C0C001823106115B9D0DF1F910F9108958F93A0
:100C1C008591803011F0E4DFFBCF8F9108958F9395
:100C2C008191803011F0DCDFFBCF8F9108958F9391
:100C3C0081E0BFDF25DC8F9108950F93880F880F1B
:100C4C00880FE82FF6E0FF1F8064B3DF08E0C8953B
:100C5C00802DC6DF31960A95D1F70F9108950404C3
:100C6C001F0404001F000C0204080E0000000C02FC
:100C7C000C020C0000001806010618001F00030CE3
:100C8C00100C03001F0004041F041F040400001FA9
:100C9C00001F001F00001515151515151500202037
:100CAC00203A2020202020202F20202F2020000040
:100CBC0070706D2000000020012002200320042011
:100CCC000520062007202020434F3232206D6F6212
:100CDC00696C65202020000020207777772E7765BF
:100CEC006967752E6C7520200000437572736F72E6
:100CFC002D506F732E203D203635000047726164F5
:100D0C00204300000F9300270093B90008E40093E0
:100D1C00B8000F9108958F9384EA8093BC00809162
:100D2C00BC0087FFFCCF9091B900987F8F910895FC
:100D3C008F938093BB0084E88093BC008091BC00AF
:100D4C0087FFFCCF9091B900987F8F91089584EC28
:100D5C008093BC008091BC0087FFFCCF8091BB00CE
:100D6C009091B900987F089584E88093BC0080919D
:100D7C00BC0087FFFCCF8091BB009091B900987F9D
:100D8C0008950F9304E90093BC000F9108950F93FD
:100D9C001F932F938F93112723E0BDDF80E0C8DFD3
:100DAC00F0DF6EDBB8DF9830C1F582E2C1DF98313D
:100DBC00A1F582E2BDDF983281F580E0B9DF98328F
:100DCC0061F588E0B5DF983241F58AE2B1DF9832FF
:100DDC0021F5D7DF5EDB5DDB9EDF9830F1F483E23B
:100DEC00A7DF9034D1F4B3DF9035B9F480930D05BF
:100DFC00AEDF903591F480930E05A9DF903569F440
:100E0C0080930F05B1DF983541F480931005B9DF5D
:100E1C0000910D05013241F001C0B3DF13952A9505
:100E2C0089F140DB3FDBB9CF10900E0500900F0528
:100E3C0080E304E6202E79D4912D00E0102E0AE0F8
:100E4C00202E73D4080E00920D05180E10920E056C
:100E5C00092E00E0102E0AE0202E67D4080E009216
:100E6C000F05180E1092100500E700931105009362
:100E7C0012050DE60093130500E2009314050027FC
:100E8C0000931505912F8F912F911F910F9108951C
:100E9C000F93882799273F9A3E9A80932A05479A61
:100EAC00469AAEDA4698ACDA4798AADAA9DA479AA3
:100EBC00A7DA469AA5DA4798A3DAA2DA4698A0DA16
:100ECC009FDA9EDA479A9CDA9BDA479899DA98DA95
:100EDC00479A96DA95DA479893DA92DA479A90DA43
:100EEC008FDA47988DDA8CDA479A8ADA89DA47985A
:100EFC0087DA86DA479A84DA83DA479881DA469A6F
:100F0C007FDA479A7DDA7CDA47987ADA469878DA8B
:100F1C00479A76DA75DA479873DA469A71DA479A0D
:100F2C006FDA6EDA47983E98469A6ADA69DA479A27
:100F3C003699FECF4798369BFECFABDA3699FECF6B
:100F4C005FDA479A5DDA5CDA36999068479858DA36
:100F5C0057DA479A55DA54DA36999064479850DA4A
:100F6C004FDA479A4DDA4CDA36999062479848DA5C
:100F7C0047DA479A45DA44DA36999061479840DA6D
:100F8C003FDA479A3DDA3CDA36999860479838DA76
:100F9C0037DA479A35DA34DA36999460479830DA8A
:100FAC002FDA479A2DDA2CDA36999260479828DA9C
:100FBC0027DA479A25DA24DA36999160479820DAAD
:100FCC001FDA1EDA1DDA1CDA3E9A469819DA479AAD
:100FDC0017DA16DA479814DA13DA3E98469A479AD3
:100FEC000FDA0EDA3699806847980ADA09DA479AE6
:100FFC0007DA06DA36998064479802DA01DA479AFA
:10100C00FFD9FED9369980624798FAD9F9D9479A0F
:10101C00F7D9F6D9369980614798F2D9F1D9479A20
:10102C00EFD9EED9369988604798EAD9E9D9479A29
:10103C00E7D9E6D9369984604798E2D9E1D9479A3D
:10104C00DFD9DED9369982604798DAD9D9D9479A4F
:10105C00D7D9D6D9369981604798D2D9D1D9D0D998
:10106C00CFD9CED93E9A469ACBD9479AC9D9C8D9A5
:10107C004798C6D98093280590932905682E792E18
:10108C00882E992E18D3822C932CA42CB52C03E5E6
:10109C00C02E0EE3D02E23D3022C132C242C352C53
:1010AC00462C572C08EE602E03E0702E78D3442487
:1010BC00552408EE602E03E0702E71D3A02CB12CB9
:1010CC00C22CD32C682E792E0FE6802E01E0902EA8
:1010DC00F2D22A183B084C085D0804EF201A0FE4E2
:1010EC00300A4F085F08022C132C242C352C00E1FD
:1010FC00402E07E2502E3ED3902D022C132C04E6EA
:10110C00202E13D3802D009117050951602E7724C2
:10111C0067FE05C0609401E0600E00932A05809084
:10112C00280590902905880C991C880C991C880C12
:10113C00991C08EE800E03E0901EBDD2022C132CDD
:10114C00242C352C08EE402E03E0502E13D304E64D
:10115C00202EEBD200912A05013039F0810D843616
:10116C0010F084569395900D07C0811987FF03C02A
:10117C0004E6800F9A959019092E1F2C0AE0202E58
:10118C00D4D200E3000E00922B0500923205100E13
:10119C0010922C05109233050CE200932D05082EAD
:1011AC001F2C0AE0202EC1D200E3000E00922E0567
:1011BC00100E10922F0505E20093300500933405B4
:1011CC00002700933105009335050F9108950F9377
:1011DC00882799273F9A3E9A479A469A11D946985A
:1011EC000FD947980DD90CD9479A0AD9469A08D9DC
:1011FC00479806D905D9469803D902D901D9479AF7
:10120C00FFD8FED84798FCD8FBD8479AF9D8F8D81D
:10121C004798F6D8F5D8479AF3D8F2D84798F0D82B
:10122C00EFD8479AEDD8ECD84798EAD8E9D8479A3E
:10123C00E7D8E6D84798E4D8E3D8479AE1D8E0D87D
:10124C004798DED8469ADCD8479ADAD8D9D8479846
:10125C00D7D8D6D8479AD4D8D3D847983E98469A58
:10126C00CFD8CED8479A3699FECF4798369BFECF2B
:10127C0010D93699FECFC4D8479AC2D8C1D836995E
:10128C0090684798BDD8BCD8479ABAD8B9D836997F
:10129C0090644798B5D8B4D8479AB2D8B1D8369993
:1012AC0090624798ADD8ACD8479AAAD8A9D83699A5
:1012BC0090614798A5D8A4D8479AA2D8A1D83699B6
:1012CC00986047989DD89CD8479A9AD899D83699BF
:1012DC009460479895D894D8479A92D891D83699D3
:1012EC00926047988DD88CD8479A8AD889D83699E5
:1012FC009160479885D884D883D882D881D83E9A73
:10130C0046987ED8479A7CD87BD8479879D878D895
:10131C003E98469A479A74D873D8369980684798FD
:10132C006FD86ED8479A6CD86BD83699806447982A
:10133C0067D866D8479A64D863D83699806247983C
:10134C005FD85ED8479A5CD85BD83699806147984D
:10135C0057D856D8479A54D853D836998860479856
:10136C004FD84ED8479A4CD84BD83699846047986A
:10137C0047D846D8479A44D843D83699826047987C
:10138C003FD83ED8479A3CD83BD83699816047988D
:10139C0037D836D835D834D833D83E9A469A30D840
:1013AC00479A2ED82DD847982BD88A5A9F40082E6A
:1013BC00192E04E6202EB9D1812D902D809316057F
:1013CC0090931705002D007831F00DE2009318056D
:1013DC009095939509C01F2C04E6202EA6D1912D33
:1013EC0000E3000E00921805092E1F2C0AE0202E97
:1013FC009CD100E3000E0092190500922205100EFC
:10140C0010921A05109223050CE200931B05082E6E
:10141C001F2C0AE0202E89D100E3000E00921C053F
:10142C00100E10921D050FED00931E050093240560
:10143C0003E400931F050093250500E200932005AB
:10144C0000932605002700932105009327050F9193
:10145C00089561DC983089F580ED6ADC983169F586
:10146C0080E066DC983249F58091360561DC983273
:10147C0021F5809137055CDC9832F9F480913805C0
:10148C0057DC9832D1F48091390552DC9832A9F4AA
:10149C0080913A054DDC983281F480913B0548DC13
:1014AC00983259F480913C0543DC983231F48091A8
:1014BC003D053EDC983209F400C063DC08952BDC5A
:1014CC00983011F09031C1F580ED32DC9831A1F5F6
:1014DC0080E02EDC983281F51EDC903169F581EDCF
:1014EC0027DC903449F533DC80933605903521F5B3
:1014FC002EDC809337059035F9F429DC8093380580
:10150C009035D1F424DC809339059035A9F41FDC97
:10151C0080933A05903581F41ADC80933B05903525
:10152C0059F415DC80933C05903531F41DDC809327
:10153C003D05983509F400C024DC08958F939F93E2
:10154C0080913A05AAD090933E0580933F059093E5
:10155C005C0580935D0590936805809369058EE228
:10156C00809340058FE280935E0580913B0595D07A
:10157C00909341058093420590935F05809360059D
:10158C0090936A0580936B058EE28093430580915E
:10159C003C0583D0909344058093450590936C054E
:1015AC0080936D0580E2809346058091380575D057
:1015BC00909347058093480590935105809352056D
:1015CC0090936205809363058AE380934905809329
:1015DC0053058091370561D090934A0580934B0554
:1015EC0090935405809355059093640580936505FD
:1015FC008AE380934C0580935605809136054DD037
:10160C0090934D0580934E05909357058093580504
:10161C00909366058093670580E280934F058093D5
:10162C00590580935A0580935B0588278093500554
:10163C008093610580936E059F918F9108950F9310
:10164C0000E00093360500E30093370502E10093B8
:10165C00380502E00093390501E000933A0505E0F6
:10166C0000933B0502E100933C0500E100933D052E
:10167C00F0DE0F9108954FDB983069F480ED58DB64
:10168C00983149F487E054DB983229F480E150DB3F
:10169C00983209F400C075DB08950F931F9300E393
:1016AC00182F807F8295800F982F812F8F70800F3D
:1016BC001F910F9108950F930FB70F930027689CFC
:1016CC001001799C2001699C300C411C501E789CA7
:1016DC00300C411C501E0F910FBF0F9108950F93AA
:1016EC000FB70F9300278C9C1001BD9C3001442434
:1016FC0055248D9C300C411C501E9C9C300C411C64
:10170C00501EAC9C400C511C601E9D9C400C511CEE
:10171C00601EBC9C500C611C701EAD9C500C611C5E
:10172C00701E0F910FBF0F9108950F930FB70F936A
:10173C0008E0000C111C10F0121410F01218039495
:10174C000A95B9F70F910FBF0F9108950F930FB72B
:10175C000F9308E0000C111C221C18F01314240425
:10176C0018F01318240803940A95A1F70F910FBFD2
:10177C000F9108950F930FB70F9300E1000C111CFC
:10178C00221C331C18F02414350418F024183508C6
:10179C0003940A9599F70F910FBF0F9108950F932A
:1017AC000FB70F9300E2000C111C221C331C441CBD
:1017BC00551C18F04614570418F046185708039493
:1017CC000A9589F70F910FBF0F91089580E1F8D119
:1017DC008DE0F6D1FED18E3321F4FBD18D3009F49E
:1017EC00089580910001816080930001089581E14A
:1017FC00E7D18DE0E5D1EDD1843469F4EAD18A33B7
:10180C0051F4E7D18C3539F4E4D18E3321F4E1D1A4
:10181C008D3009F40895809100018160809300015E
:10182C00089580E9CDD18DE0CBD1D3D18E3321F485
:10183C00D0D18D3009F4089580910001816080939E
:10184C000001089581E9BCD18DE0BAD1C2D18E33AB
:10185C0021F4BFD18D3009F408958091000181608D
:10186C0080930001089584E1ABD180E2A9D18091ED
:10187C000101A6D180910201A3D180910301A0D1D5
:10188C008DE09ED1A6D18E3321F4A3D18D3009F4F5
:10189C00089580910001816080930001089590D19A
:1018AC0098D18E3321F495D18D3009F4089580911F
:1018BC00000181608093000108958DE081D189D170
:1018CC008E3329F486D18D3061F481E008958E3405
:1018DC0041F47FD1843429F47CD18D3011F480E033
:1018EC00089580910001816080930001089583E147
:1018FC0067D18DE065D16DD16CD16BD16AD169D1D5
:10190C0068D167D18093040164D18093050161D1C2
:10191C0060D1809306015DD1809307015AD18093E9
:10192C00080157D18093090154D180930A0151D1F8
:10193C0080930B014ED180930C014BD14AD149D1EC
:10194C0048D147D146D145D180930D0142D141D1E7
:10195C0080930E013ED180930F013BD13AD139D106
:10196C008E3321F436D18D3009F408958091000125
:10197C00816080930001089585E422D18DE020D10F
:10198C0028D1853421F425D18D3009F40895809126
:10199C0000018160809300010895089585E610D1BF
:1019AC008DE00ED116D1853621F413D18D3009F48A
:1019BC000895809100018160809300010895AF9398
:1019CC00BF93882780930002A1E0B2E081E0F8D0B9
:1019DC008DE0F6D0FED0FDD08D93AA23A1F08D30F2
:1019EC0031F480910002839580930002F4CF8E3302
:1019FC0091F7EFD08D3009F40BC08091000181601C
:101A0C008093000105C080910001826080930001E9
:101A1C00BF91AF910895AF93BF93A2E1B1E081E084
:101A2C00CFD080E2CDD08D91CBD08D30E1F7D1D01D
:101A3C00D0D08032E9F7CDD080931F01CAD08093EB
:101A4C002001C7D080932101C4D080932201C1D042
:101A5C00C0D08E3331F4BDD08D3019F4BF91AF911D
:101A6C00089580910001816080930001BF91AF9136
:101A7C000895AF93BF93A2E1B1E089E0A1D080E2D9
:101A8C009FD08D919DD08D30E1F7A3D08E3331F462
:101A9C00A0D08D3019F4BF91AF91089580910001C1
:101AAC00816080930001BF91AF910895AF93BF9374
:101ABC00A0E0B3E088E084D080E282D0882780D098
:101ACC007FD07ED0809110017BD08DE079D08D912C
:101ADC0077D080911001A817D1F77BD08E3331F4D9
:101AEC0078D08D3019F4BF91AF9108958091000199
:101AFC00816080930001BF91AF910895AF93BF9324
:101B0C00A2E1B1E08AE05CD080E25AD08D9158D04D
:101B1C008D30E1F75ED08E3331F45BD08D3019F41B
:101B2C00BF91AF9108958091000181608093000175
:101B3C00BF91AF910895AF93BF93A2E1B1E08EE056
:101B4C003FD080E23DD08D913BD08D30E1F741D03C
:101B5C008E3331F43ED08D3019F4BF91AF9108958E
:101B6C0080910001816080930001BF91AF91089535
:101B7C00AF93BF93A0E0B4E08BE022D080E220D002
:101B8C0088271ED01DD01CD08091110119D08DE05A
:101B9C0017D01FD08D9380911101A817D1F719D0B0
:101BAC008E3331F416D08D3019F4BF91AF91089566
:101BBC0080910001816080930001BF91AF910895E5
:101BCC009F939091C80095FFFCCF8093CE009F917E
:101BDC0008958091C80087FFFCCF8091C8008C715C
:101BEC0019F48091CE00089580930001089544412A
:101BFC0054554D095A4549540954454D5045524187
:101C0C00545552205BC2B0435D0946455543485478
:101C1C0049474B454954205B255D09433032205BD5
:101C2C0070706D5D0D0D000020205F20205F202066
:061C3C002E7478740D0007
:00000001FF
